S110C000FC7FFE1A831040260CCC4F4EFD31
S111C00D7FFE8E7F6A7E1040B610208A03B735
S111C01B1020B6B7FF81052206810125022000
S110C029028603B7102B4FB7102C860CB7FE
S111C036102DCED715B6102E2AFBA600270615
S111C04408B7102F20F14FB77FBDB17FBD2686
S111C052F743B77FBDB17FBD26EECED720B633
S111C060102E2AFBA600270608B7102F20F189
S111C06E8E7FAC7F7FBCB6B7FF8105220681B2
S111C07C01250220028603B7102B4FB7102CAB
S111C08A860CB7102D4FCE7FADC60CA7000854
S111C0985A26FAFE7FFE8C4F4E27288C10404D
S111C0A62723CE4F4EFF7FFECED748BDCB9250
S111C0B48601B77FBB7F7FBA4FC60ECE7FC01A
S110C0C2A700085A26FABDCAD0CED998BDF1
S110C0CFCB92BDCAD084DFCEC0DEC605BD55
S10FC0DCCA8A20444D4F5257C0CBC0F01C
S109C0E8C2E2C607C925EF
S10CC0EECBA0CEDB06BDCB92CE43
S10CC0F77FC2BDCB92CEDBA1BDDA
S110C100CB92BDCAD084DFCEC10FC604BDF2
S10EC10DCA8A20444D491BC0F0C11E2B
S10AC118C132C213C0CBCEFB
S10EC11FDBE0BDCB92CE7FC0860CB7E6
S10CC12A7FC0BDCADB7EC0F07FBA
S10DC1337FBCCEDBB4BDCB920FBD80
S111C13DCAD0811B26037EC06E815326F2BD3C
S111C14BCAD08139276D813126E7CE7FCF4FD0
S111C159A7048602A701BDCAD0A702BDCAD0A2
S111C167A703BDC9DB8003B77FBDCE7FCF4FDA
S111C175A7068604A701BDCAD0A702BDCAD082
S110C183A703BDCAD0A704BDCAD0A705BD3F
S111C190CA1E188FCE7FCF4FA7048602A701C8
S111C19EBDCAD0A702BDCAD0A703BDC9DB1815
S110C1ACA70018087A7FBD26DFBDCAD0BDEC
S111C1B9CAD07EC13CCE7FCF4FA7048602A71A
S111C1C701BDCAD0A702BDCAD0A703BDC9DB03
S10DC1D5B77FBDBDCAD0BDCAD07A41
S111C1DF7FBD26F5CE0002BDCA78CEDB06FF7A
S10CC1ED7FBECED715BDC8C8FC05
S111C1F67FD01A83FC9B2712CE000ABDCA78A4
S10DC204CEF096BDCB92BDCAD0BDAA
S10CC20ECAD07EC06E7F7FBCCE55
S111C217DBB4BDCB920FBDCAD0811B26037EC3
S111C225C06E813A26F2CE7FCF4FA704860268
S110C233A701BDCAD0A702BDCAD0A703BD94
S111C240C9DBB77FBDCE7FCF4FA7068604A70C
S111C24E01BDCAD0A702BDCAD0A703BDCAD085
S110C25CA704BDCAD0A705BDCA1E188FCE09
S111C2697FCF4FA7048602A701BDCAD0A7024B
S111C277BDCAD0A703BDC9DB4D262ACE7FCF9A
S110C2854FA7048602A701BDCAD0A702BDC1
S110C292CAD0A703BDC9DB18A70018087A9D
S10EC29F7FBD26DFBDCAD0BDCAD07E23
S10FC2AAC21DBDCAD0BDCAD0CE0002BD6A
S10CC2B6CA78CEDB06FF7FBECE80
S111C2BFD715BDC8C8FC7FD01A83FC9B27127C
S110C2CDCE000ABDCA78CEF096BDCB92BD5E
S10CC2DACAD0BDCAD07EC06ECEEC
S10EC2E3DC70BDCB92BDCAD084DFCE5E
S110C2EEC2F5C605BDCA8A204445464D1B55
S109C2FBC2E2C307C3EE1A
S10AC301C449C586C0CBCE80
S110C308DD4DBDCB92CE7FCF8604A700BDD6
S111C315CADB6D0126037EC2E2BDCA1E2407E8
S111C3238607BDCB5120DDCED734BDCB92BDF5
S111C331CA6BBDCA6B8FBDCA6B18CE00103C20
S111C33FCED72FBDCB92383C8F3837BDCA6B9A
S111C34D368620BDCB5132BDCAA7BDCB5117D9
S10FC35BBDCB5132BDCAA7BDCB5117BDEC
S10FC367CB518609BDCB513CCED72BBD79
S110C373CB9238C610A6000837BDCAA7BD7E
S111C380CB5117BDCB518620BDCB5133C10923
S111C38E260A8620BDCB518620BDCB515A26EF
S111C39CDB8F8300108FC6108620BDCB518628
S111C3AA20BDCB51A6000881202509817E22EA
S111C3B805BDCB512005862EBDCB515A26E87B
S111C3C6180927037EC33E3CCEDDABBDCB92EF
S110C3D438BDCAD081202707812D27077EA0
S111C3E1C0CB8F7EC32A8F8302007EC32ACE78
S10CC3EFDDE7BDCB92CEDE8ABD70
S111C3F8CB92CE7FCF8604A700BDCADBA60180
S111C40626037EC0CB81012619A60284DF81A5
S111C4144E262A183C38088608BDCB513C320F
S111C42233BDCB852008BDCA1E25143736381D
S111C4303C1838A600CEDE9CBDCB92BDCB7668
S10FC43E7EC3F48607BDCB517EC3EECE56
S10EC44ADEA5BDCB92BDCAD084DFCEBE
S110C455C45CC603BDCA8A2046431BC4490B
S10AC462C468C4F4C2E2CE79
S110C469DF13BDCB92CE7FCF8604A700BDAC
S111C476CADB6D01260A7EC2E28607BDCB51E9
S111C48420E2BDCA1E25F437361838CEDF5527
S111C492BDCB92CE7FCF8604A700BDCADB6D62
S111C4A001260A7EC4498607BDCB5120E2BDA9
S10EC4AECA1E25F4FD7FBECEDF8CBD4E
S111C4B9CB92CE7FCF8602A700BDCADB6D01F9
S110C4C7260A7EC4498607BDCB5120E2BD84
S111C4D4C9DB25F4183C38BC7FBE2205A70046
S110C4E20820F6CEDFB5BDCB92CE000ABD1A
S10CC4EFCA787EC0CBCEDFC7BDC4
S111C4F8CB92CE7FCF8604A700BDCADB6D01B8
S110C506260A7EC2E28607BDCB5120E2BDAD
S111C513CA1E25F437361838CEE009BDCB9287
S111C521CE7FCF8604A700BDCADB6D01260ABB
S111C52F7EC4498607BDCB5120E2BDCA1E253D
S10EC53DF4FD7FBECEE040BDCB92CEEB
S111C5487FCF8604A700BDCADB6D01260A7EE4
S111C556C4498607BDCB5120E2BDCA1E25F4A0
S111C56437363818BC7FBE220A18A600180805
S111C572A7000820F0CEE077BDCB92CE000AE1
S10DC580BDCA787EC0CBCEE089BDB1
S10CC58ACB92CEE132BDCB92CE7E
S111C5937FCF8604A700BDCADBA601260A7E60
S111C5A1C0CB8607BDCB5120DC81012619A634
S111C5AF0284DF814E26ED183C38088608BD54
S111C5BDCB513C3233BDCB852008BDCA1E25B0
S111C5CBD73736383C1838CEE141BDCB92CE7E
S111C5D97FCF8602A700BDCADB6D0126107E4F
S10EC5E7C2E28607BDCB51CEE150BD7F
S110C5F2CB9220DCBDC9DB25EE18A700CEDE
S10CC5FFE14ABDCB927EC58CCE4D
S10EC608E156BDCB92BDCAD084DFCE4A
S110C613C61AC605BDCA8A20435645521BEF
S109C620C607C62CC64A41
S10DC626C69DC85CC0CBCC0000FD2B
S111C6307FFE0FCCC000FD7FFCB610398A08D7
S110C63EB7103907847F0601CF7EC06ECE91
S111C64BE1FEBDCB92FC7FFE1A834F4E260308
S10DC659CCC000CED72FBDCB92BD9C
S10CC663CB85CED72BBDCB92CEC2
S110C66CE20818CE7FD4C61437C61B3ABDB1
S111C679CB92C602183A18EC003CCED72FBD67
S10CC687CB92BDCB85CED72BBDAF
S111C690CB9238335A26DDBDCAD07EC0CBCE45
S10EC69EE43FBDCB92BDCAD084DFCEC8
S110C6A9C6B0C605BDCA8A20454257531BC2
S109C6B6C69DC6C2C71BAD
S10AC6BCC765C7E3C0CBCE44
S110C6C3E4EBBDCB92CE7FCF8604A700BD73
S111C6D0CADB6D0126037EC69DBDCA1E24076B
S111C6DE8607BDCB5120DD8FB610398A40B7D8
S111C6EC10398616B7103BA7008617B7103B0F
S111C6FA0FCE0001BDCA787F103BB610398404
S111C708BFB71039CEE584BDCB92CE0005BD7F
S10CC716CA787EC69DCEE559BD2A
S111C71FCB92BDCAD081592707817927037EAA
S110C72DC69DB610398A40B710398606B78C
S111C73A103BB7B6008607B7103B0FCE0001C8
S111C748BDCA787F103BB6103984BFB71039D4
S110C756CEE584BDCB92CE000ABDCA787E2C
S10CC763C69DCEE522BDCB92CEA9
S111C76C7FCF8604A700BDCADB6D0126037EC5
S111C77AC69DBDCA1E24078607BDCB5120DD17
S111C788188FCEE596BDCB92CE7FCF8602A74A
S111C79600BDCADB6D01260A7EC69D8607BD66
S111C7A4CB5120E2BDC9DB25F4F61039CA40A2
S111C7B2F71039C602F7103B18A7008603B72C
S110C7C0103B0FCE0001BDCA787F103BB6C0
S111C7CD103984BFB71039CEE584BDCB92CEAF
S10FC7DB0005BDCA787EC69DCEE5C3BD36
S111C7E7CB92BDCAD0811B260A7EC06E860787
S111C7F5BDCB5120E9813125F5813522F1803B
S111C80330F61039CA40F71039C616F7103B4C
S110C811B7B7FFC617F7103B0FCE0001BDEF
S111C81ECA787F103BF61039C4BFF71039C634
S111C82C02F7103BB7B7FF8603B7103B0FCEE1
S111C83A0001BDCA787F103BB6103984BFB729
S111C8481039CEE68DBDCB92CE0005BDCA7868
S10DC856BDCAD07EC06ECEE6D7BD89
S111C860CB92CE7FCF8604A700BDCADB6D014C
S111C86E26078607BDCB5120E5BDCA1E240255
S111C87C20F2188FCEE73DBDCB92CE7FCF8643
S110C88A04A700BDCADB6D0126078607BDAB
S111C897CB5120E5BDCA1E240220F2FD7FBE57
S111C8A5183C38860ABDCB51BDC8C8CEE76F1B
S10DC8B3BDCB92FC7FD0BDCB85CE37
S10CC8BDE7A2BDCB92BDCAD07EF6
S111C8C6C06E18CEF14ECC0000FD7FD086016E
S110C8D4B77FBDA600B47FBD27028601F624
S111C8E17FD1C47F183C183A18E6001838F7C7
S10FC8EF7FCFB87FCFF67FD0595959F79E
S10DC8FB7FCFB87FCF44797FD17955
S111C9057FD0747FBD25098601B17FBD27094F
S111C91320C28680B77FBD20BBBC7FBE270339
S111C9210820B339CEE7CBBDCB92BDCAD0847B
S110C92FDFCEC938C603BDCA8A2050531B91
S109C93CC925C944C985A8
S10CC942C0CBCEE82DBDCB92CE92
S111C94B7FCF8604A700BDCADB6D0126037EE4
S10EC959C0CBBDCA1E251ECEE867BD82
S111C964CB92CE0001BDCA78CE10403C1838EC
S111C9728E7F6A7F7FBC3736CC000039860783
S10FC980BDCB5120BFCEE888BDCB92CEC9
S111C98C7FCF8604A700BDCADB6D0126037EA3
S10EC99AC0CBBDCA1E2519CEE867BD46
S111C9A5CB928E7F6ACEC9B43C3736CC0000EC
S111C9B339BDCAD07EC0CB8607BDCB5120C48F
S111C9C180308109230484DF8007C030C1095F
S111C9CF2304C4DFC007484848481B393CA66F
S111C9DD01810226390808A600272281302590
S111C9EB2F81392F0C84DF8141252581462FB1
S111C9F909201F8030A7000820E18037A70026
S111CA070820DA0909A600080848484848092A
S111CA15AA00080C38390D38393CA6018104FA
S111CA2326430808A6002722813025398139D0
S111CA312F0C84DF8141252F81462F092029F7
S111CA3F8030A7000820E18037A7000820DA25
S111CA4D09090909A6004848484808AA000833
S111CA5BE6000858585858EA00080C38390FFD
S111CA69383936860ABDCB51860DBDCB51320D
S111CA77393C183C18CE37CD180926FC092688
S111CA85F51838383931313C18383A08183C65
S111CA93183A18A100183827055A270320F076
S111CAA1583AEE006E003C36CECAC01654540D
S111CAAF54543AE60017CECAC033C40F3AE618
S111CABD0038393031323334353637383941A8
S110CACB4243444546B6102E842027F9B698
S111CAD8102F3936373C183CE60008083C188D
S111CAE638183A5FBDCAD0811B27528108263A
S111CAF4135D27F2BDCB518620BDCB518608C1
S111CB02BDCB515A20E2810D260F09E7000831
S111CB103C3A6F00381838383332398120250A
S111CB1E1D817E22193C3A183C1830CDAC0023
S111CB2C183838270B3C3AA700385CBDCB51B3
S111CB3A20AE8607BDCB5120A75F09E7000897
S111CB483A6F0018383833323936B6102E2AB8
S110CB56FB32B7102F3936373C5F8620BD07
S111CB63CB513C3AA60038BDCB765CC105260A
S111CB71EE383332393637BDCAA7BDCB511763
S111CB7FBDCB513332393637BDCB763236BD9D
S111CB8DCB76333239363CA6002705088DB628
S111CB9B20F7383239B610208A03B7102086EE
S111CBA908B7100B7D7FBC264A8601B77FBCFF
S10DCBB7CED00BFF7FF8CED094FF20
S111CBC17FF418CE7F6ACE1040860318081841
S111CBCF091809CDEF004A26F65F8602180900
S111CBDD18E7004A26F886D0180918A7001891
S110CBEB0918FF7F6B200ABDCFB62008BDDE
S10ECBF8CEB72003BDCEB17F7FBA7F13
S10CCC037FB9CEE930BDCB92BD2E
S111CC0CCAD084DFCECC18C60DBDCA8A205013
S111CC1A585941424E53431B5254474DCBFCD4
S109CC28CC42CC6DCC9857
S109CC2ECCC3CCEECD19CD
S109CC34CD42CDDAC0CBB5
S109CC3ACE36CE4CCE47BD
S10CCC40CEA0CEEE37BDCB92CE9E
S111CC497FCF8604A700BDCADB6D0126037EE3
S111CC57CBF7BDCA1E24078607BDCB5120DDD6
S10FCC65FE7F6BED087ECBF7CEEE61BDC8
S111CC71CB92CE7FCF8604A700BDCADB6D0137
S110CC7F26037ECBF7BDCA1E24078607BD21
S110CC8CCB5120DDFE7F6BED047ECBF7CE97
S110CC99EE4CBDCB92CE7FCF8604A700BD2C
S111CCA6CADB6D0126037ECBF7BDCA1E240730
S110CCB48607BDCB5120DDFE7F6BED067EB3
S10CCCC1CBF7CEEE78BDCB92CE88
S111CCCA7FCF8602A700BDCADB6D0126037E64
S111CCD8CBF7BDC9DB24078607BDCB5120DD99
S10FCCE6FE7F6BA7037ECBF7CEEE8DBD66
S111CCF2CB92CE7FCF8602A700BDCADB6D01B8
S110CD0026037ECBF7BDC9DB24078607BDE3
S110CD0DCB5120DDFE7F6BA7027ECBF7CE5D
S110CD1AEEA4BDCB92CE7FCF8602A700BD54
S111CD27CADB6D0126037ECBF7BDC9DB2407F2
S111CD358607BDCB5120DDB77FBB7ECBF7CE8A
S10ECD437FF8CCD00BED00CEE904BD5E
S111CD4ECB92BDCAD0811B26037ECBF280316E
S111CD5C16B77FBD810323078607BDCB512088
S111CD6ADFCE7FAD583A1AEE0027138607BDC0
S10FCD78CB51CEE958BDCB92CE000ABDD1
S10ECD84CA7820C2CEE8C4BDCB92CE1A
S111CD8F7FCF8604A700BDCADB6D0126037E9C
S110CD9DCBF2BDCA1E2523188FF67FBDCE34
S111CDAA7FB53A18A600A700864118A7001806
S110CDB8A100260BCE7FAD583A1AEF007E85
S10ECDC5CBF28607BDCB51CEE9B0BD18
S111CDD0CB92CE0014BDCA7820AECE7FF8CC34
S10ECDDED00BED00CEE904BDCB92BDEC
S111CDE9CAD0811B26037ECBF2803116810353
S111CDF723078607BDCB5120E2CE7FAD583A0C
S111CE051AEE0026138607BDCB51CEE984BD7C
S111CE13CB92CE0014BDCA7820C554CE7FB594
S111CE213AA60018A700CE7FAD18CE00005828
S111CE2F3A1AEF007ECBF2CEE9E2BDCB92CEF2
S110CE3D0001BDCA780FBE7F6B3B8639B77C
S111CE4A7FB9FE7F6B1AEE0818A60081412600
S111CE580FCEEF88BDCB92CE001EBDCA787EF1
S111CE66CBFC8639B17FB9261418A100260F23
S110CE74CEF058BDCB92CE000FBDCA787E23
S110CE81CBFC0FC631FE100E3AFF101EB69A
S111CE8E102084FEB71020BE7F6B30A60084F7
S111CE9CBFA7003BB67FBBB77FBA27064AB7D5
S10ECEAA7FBA209E7ECBFFCEE9FFBDC7
S10DCEB5CB9218FE7F6BCEED27BD73
S10FCEBFCB9218EC08BDCB85CEED32BD43
S10DCECBCB928FBDCB5CCEEDC1BD50
S10FCED5CB92CDEE08BDD0D4CEED3DBD17
S110CEE1CB92183C38C6093A8FBDCB85CEE4
S10DCEEEED48BDCB928FBDCB5CCEA6
S10FCEF8ED53BDCB9218EC06BDCB85CEEB
S10DCF04ED5EBDCB928FBDCB5CCE79
S10FCF0EED69BDCB9218EC04BDCB85CEC0
S10DCF1AED75BDCB928FBDCB5CCE4C
S10FCF24ED8DBDCB9218A602BDCB76CEDD
S10FCF30ED81BDCB9218A603BDCB76CEDC
S10CCF3CEDB4BDCB92B67FBBBD80
S10FCF45CB76CEED9ABDCB9218A601BDB0
S111CF51CB76CEEDA7BDCB9218A60144444486
S110CF5F4424078631BDCB5120058630BD2A
S111CF6CCB518620BDCB5118A6014444442469
S111CF7A078631BDCB5120058630BDCB5186D4
S111CF8820BDCB5118A601444424078631BDB8
S111CF96CB5120058630BDCB518620BDCB513A
S111CFA418A6014424078631BDCB5120058612
S10FCFB230BDCB5118CE7FADCEEDD3BD09
S111CFBECB9218EC00180818081A83000027FC
S111CFCC03BDCB85CEEDECBDCB9218EC001866
S110CFDA0818081A8300002703BDCB85CE7C
S111CFE7EE05BDCB9218EC00180818081A834A
S111CFF500002703BDCB85CEEE1EBDCB9218E7
S111D003EC002703BDCB8539B610208A03B795
S110D01110208608B7100BBF7F6B8601B797
S111D01E7FBC3018308E7FAC18A6008410261C
S110D02C090E3CCEF07FBDCB9238EC07CE50
S111D0397FAD188F4F1AAC00272008084C81D9
S111D04704270220F2CEEEBBBDCB92188FBDA3
S10CD055CB85CEEF16BDCB92BDD4
S111D05ECAD07ECBFC6F006F01CE7FB5163AB0
S111D06CA60018A700CEEF38BDCB92178B316B
S10FD07ABDCB51CEEF54BDCB92188FBD3E
S10CD086CB85CEEF66BDCB92BD53
S111D08FCAD07ECBFCB610208A03B7102086D0
S111D09D08B7100BBF7F6B18308E7FAC18A63F
S111D0AB00841026090E3CCEF07FBDCB9238D7
S111D0B98601B77FBC7D7FBA27067A7FBA7ED8
S10ED0C7CE4C7D7FB927037ECE4C7E4B
S111D0D2CBF7A600C6008118270A811A27058D
S111D0E081CD26045C5C5C08FF7FCFF77FD116
S111D0EEA600B77FD208FF7FCF815F230F819A
S111D0FC8D270B818F270781CF27037ED1B1AB
S111D10AF67FD1C1022504BDD38D39F67FD244
S111D1185FBDD2A95D2604BDD38D39B67FD28A
S111D126818D2604C605200A818F270481CF3F
S111D1342605C601BDD2A9F67FD3C101261A75
S110D142F67FD1C100270FB67FD2C602BD13
S111D14FD2A95D2604BDD38D39BDD2CE39F6EA
S111D15D7FD3C10526107D7FD12704BDD38D5D
S111D16B39BDD2CEBDD30C39F67FD3C1112706
S111D17904C11026117D7FD12704BDD38D394A
S10FD187BDD2CEBDD3632006BDD2CEBD08
S110D193D2EF8620BDCB51BDD3638620BDF5
S111D1A0CB51F67FD3C10D2704C1102603BD69
S111D1AED30C39817F222CF67FD1C1022504D7
S111D1BCBDD38D39846F5FBDD2A95D2604BD3D
S111D1CAD38D39BDD2CEB67FD284F0816026DB
S111D1D804BDD2EF39BDD3703981872704819D
S111D1E6C72604BDD38D3984CF5FBDD2A95DA9
S111D1F42604BDD38D39B67FD284CF818D261B
S111D20204C6072016818F2604C607200E815D
S111D210CF2604C60A20068183260CC608BD5C
S111D21ED2A95D2604BDD38D39F67FD3C1039A
S111D22C2708C1072704C1082636B67FD2841E
S111D23ACF81832611F67FD1C102250AC60FCB
S111D248BDD2A9C608F77FD3F67FD1C1012756
S111D25604C103260DB67FD284B081A0270444
S111D264BDD38D39BDD32639F67FD1C1012744
S111D27204C1022615B67FD284CFF67FD3C145
S110D280092604C60B2002C60CBDD2A9F677
S111D28D7FD1C102250DB67FD284B081A027C7
S111D29B04BDD38D39C608F77FD3BDD3263921
S111D2A9CED396A10426115D2704E105260AC2
S111D2B7E605F77FD3FF7FD45C3937C6063A0D
S111D2C5E600C1043326E05F39FE7FD4A600E4
S111D2D3BDCB51A601BDCB51A602BDCB51A6C9
S111D2E10381202705BDCB518620BDCB5139DA
S111D2EFBDD363862CBDCB51F67FD1C1012780
S111D2FD04C1032604865920028658BDCB5175
S111D30B39FE7FCFE60008FF7FCF5D2B033A8B
S111D3192004095C26FC3C3233BDCB8539BDB3
S111D327D2CEB67FD284B08180261D8623BD6F
S111D335CB51BDD363F67FD3C108270139FE67
S111D3437FCFA600BDCB7608FF7FCF39819047
S111D3512604BDD3633981A02604BDD2EF3972
S111D35FBDD37039FE7FCFA600BDCB7608FF8C
S111D36D7FCF39FE7FCFEC00BDCB850808FFD3
S111D37B7FCF39496C6C6567616C204F70631D
S111D3896F6465003CCED37EBDCB9238394133
S111D3974241201B01414258203A01414259B3
S111D3A5203A0241444341890341444342C9B2
S111D3B303414444418B0341444442CB0341B3
S111D3C1444444C308414E44418403414E4455
S111D3CF42C40341534C20680441534C41486E
S111D3DD0141534C42580141534C4405014157
S111D3EB5352206704415352414701415352AB
S111D3F942570142434320240542434C521D37
S111D4070E424353202505424551202705427D
S111D4154745202C05424754202E0542484925
S111D4232022054248532024054249544185E5
S111D4310342495442C503424C45202F054294
S111D43F4C4F202505424C53202305424C54EB
S111D44D202D05424D49202B05424E45202638
S111D45B0542504C202A054252412020054231
S111D46952434C1F0D42524E20210542525395
S111D477451E0D425345541C0E425352208D47
S111D4850542564320280542565320290543EC
S111D4934241201101434C43200C01434C49FB
S111D4A1200E01434C52206F04434C52414F65
S111D4AF01434C52425F01434C56200A014394
S111D4BD4D50418103434D5042C103434F4D36
S111D4CB206304434F4D414301434F4D4253F0
S111D4D90143504420830F435058208C0943D4
S111D4E75059208C0B44414120190144454307
S111D4F5206A04444543414A01444543425AD7
S111D503014445532034014445582009014495
S111D5114559200902454F52418803454F52A7
S111D51F42C803464449560301494449560292
S111D52D01494E43206C04494E43414C0149D0
S111D53B4E43425C01494E53203101494E5883
S111D549200801494E592008024A4D50206E18
S111D557044A5352208D074C44414186034C34
S111D565444142C6034C444420CC084C445379
S111D573208E084C445820CE094C445920CE3A
S111D5810B4C534C2068044C534C4148014C55
S111D58F534C4258014C534C4405014C53522A
S111D59D2064044C53524144014C53524254F6
S111D5AB014C53524404014D554C203D014E99
S111D5B945472060044E45474140014E45471A
S111D5C74250014E4F502001014F5241418A03
S111D5D5034F524142CA03505348413601509D
S111D5E35348423701505348583C01505348B6
S111D5F1593C0250554C41320150554C4233C6
S111D5FF0150554C58380150554C59380252C1
S111D60D4F4C206904524F4C414901524F4C7E
S111D61B425901524F52206604524F5241466A
S111D62901524F52425601525449203B0152C5
S111D637545320390153424120100153424301
S111D64541820353424342C203534543200D26
S111D65301534549200F01534556200B015346
S111D661544141870753544142C70753544470
S111D66F20CD0753544F50CF01535453208FF6
S111D67D0753545820CF0A53545920CF0C534E
S111D68B554241800353554242C00353554259
S111D699448308535749203F01544142201650
S111D6A7015441502006015442412017015401
S111D6B550412007015445535400015453546E
S111D6C3206D04545354414D01545354425DA0
S111D6D1015453582030015453592030025450
S111D6DF585320350154595320350257414900
S111D6ED203E01584744588F01584744598F36
S111D6FB024252534512104252434C13104245
S111D709534554141142434C5215110453431A
S111D71749202D204F4B0D0A0052414D202D6C
S111D725204F4B0D0A001B5B6D001B5B316D2A
S111D73300201B5B324A1B5B303B30481B5B03
S111D7416D001B5B376D001B5B324A1B5B31B6
S111D74F6D1B5B33336D1B5B34366D1B5B321D
S111D75D3B32344820C9CDCDCDCDCDCDCDCD80
S111D76BCDCDCDCDCDCDCDCDCDCDCDCDCDCD76
S111D779CDCDCDCDCDCDBB201B5B333B3234AB
S111D7874820BA20202020434F4D50555445D1
S111D7955220454E47494E454552494E4720C5
S111D7A3202020BA201B5B34306D201B5B3429
S111D7B1366D1B5B343B32344820BA202020F6
S111D7BF202020202020544543484E4F4C4F3C
S111D7CD4759202020202020202020BA201B95
S111D7DB5B34306D201B5B34366D1B5B353BBD
S111D7E932344820BA20202020202020202086
S111D7F7204D6963726F3131202020202020E4
S111D8052020202020BA201B5B34306D201B15
S111D8135B34366D1B5B363B32344820BA2042
S111D8212020363848433131204D6F6E697433
S111D82F6F722050726F6772616D202020BAF4
S111D83D201B5B34306D201B5B34366D1B5B8F
S111D84B373B32344820C8CDCDCDCDCDCDCD28
S111D859CDCDCDCDCDCDCDCDCDCDCDCDCDCD87
S111D867CDCDCDCDCDCDCDBC201B5B34306DF1
S111D875201B5B383B32354820202020202029
S111D8832020202020202020202020202020D3
S111D8912020202020202020202020201B5B8F
S111D89F6D1B5B31313B33354857726974742D
S111D8AD656E2062793A1B5B31323B333248A0
S111D8BB4772616E7420502E204265617474B1
S111D8C969651B5B31353B3333484D61726337
S111D8D7682020312C20313939361B5B313763
S111D8E53B33344856657273696F6E20312EE2
S111D8F330351B5B376D1B5B31393B333448DA
S111D901436F70797269676874203139393662
S111D90F1B5B32303B333048416C6C20526954
S111D91D676874732052657365727665641BC7
S111D92B5B6D1B5B32323B31374857686174C9
S111D939207368616C6C2069742070726F66D4
S111D94769742061206D616E20696620686538
S111D955206761696E657468206120686967E7
S111D963681B5B32333B3139486C6576656C6A
S111D971206C616E67756167652C20627574A9
S111D97F206C6F7365207369676874206F668F
S111D98D2068697320636F64653F00201B5B94
S111D99B324A1B5B6D1B5B316D1B5B376D1BD2
S111D9A95B323B323548434F4D505554455286
S111D9B720454E47494E454552494E4720549F
S111D9C54543484E4F4C4F47591B5B6D1B5B4F
S111D9D3316D1B5B353B3234484D6963726F16
S111D9E13131202D20363848433131204D6F2E
S111D9EF6E69746F722050726F6772616D1BE7
S111D9FD5B373B3335484D61696E204D656ED6
S111DA0B751B5B31303B323248441B5B6D6F40
S111DA19776E6C6F6164094D6F746F726F6C81
S111DA2761206F7220496E74656C204865782A
S111DA352046696C651B5B316D1B5B31313B18
S111DA433232484D1B5B6D656D6F727909447C
S111DA51756D702C204578616D696E652C2012
S111DA5F46696C6C2C204D6F646966791B5B04
S111DA6D316D1B5B31323B3232484F1B5B6D17
S111DA7B7074696F6E7309436F6C6420426FA0
S111DA896F742C20566563746F72732C2052D8
S111DA976F6D20546573741B5B316D1B5B3126
S111DAA5333B323248521B5B6D756E09507272
S111DAB36F6772616D206F7220537562726F1F
S111DAC17574696E651B5B316D1B5B31343B04
S111DACF323248571B5B6D696E646F770954E1
S111DADD726163652F427265616B706F696ED2
S111DAEB742057696E646F771B5B31373B33D1
S111DAF9354853656C656374696F6E3F001B9E
S111DB075B373B3333481B5B4A1B5B6D1B5B78
S111DB15316D446F776E6C6F6164204D656EE8
S111DB23751B5B31303B3235484D1B5B6D6F1B
S111DB31746F726F6C6120532D5265636F72B6
S111DB3F641B5B316D1B5B31323B3235484950
S111DB4D1B5B6D6E74656C204865782046691C
S111DB5B6C651B5B31343B3235481B5B316D0E
S111DB69441B5B6D656661756C7420446F77B8
S111DB776E6C6F61642046696C65204E616DB2
S111DB85651B5B31353B32394843757272655E
S111DB936E742066696C656E616D653A2000E3
S111DBA11B5B31383B33354853656C65637448
S111DBAF696F6E3F001B5B31383B3239481BF7
S111DBBD5B4B1B5B316D48433131205761696E
S111DBCB74696E6720666F722046696C65206F
S111DBD92E2E2E1B5B6D001B5B31303B323554
S111DBE7481B5B4A1B5B31333B32354850729E
S111DBF56F636F6D6D206C6F6F6B73206F6EBE
S111DC03207468652073637265656E20666F19
S111DC117220746578741B5B31343B323548E5
S111DC1F746F2075736520617320612066693F
S111DC2D6C656E616D652E1B5B31363B3235C6
S111DC3B485573652074686520666F726D200D
S111DC4946494C454E414D452E455854203A0F
S111DC571B5B376D2020202020202020202061
S111DC6520201B5B31363B353248001B5B37F9
S111DC733B3333481B5B4A1B5B6D1B5B316DFF
S111DC81204D656D6F7279204D656E751B5BCD
S111DC8F31303B323548441B5B6D756D7009B6
S111DC9D202020446973706C6179204D656D00
S111DCAB6F727920426C6F636B1B5B316D1BD3
S111DCB95B31313B323548451B5B6D78616D44
S111DCC7696E6509202020496E6469766964DF
S111DCD575616C204C6F636174696F6E731B14
S111DCE35B316D1B5B31323B323548461B5BB7
S111DCF16D696C6C2F436F707920204D656D4A
S111DCFF6F727920426C6F636B1B5B316D1B7F
S111DD0D5B31333B3235484D1B5B6D6F6469EF
S111DD1B6679092020204D656D6F72792F52B4
S111DD2965676973746572204C6F6361746979
S111DD376F6E731B5B31373B33354853656C9D
S111DD45656374696F6E3F001B5B31303B32C7
S111DD5335481B5B4A1B5B6D1B5B31323B3357
S111DD613048446973706C6179204D656D6FB4
S111DD6F727920426C6F636B1B5B31343B3264
S111DD7D3748456E7465722053746172746980
S111DD8B6E6720416464726573733A201B5BFB
S111DD996D1B5B376D202020201B5B31343B5B
S111DDA7353148000A0D0A0D09535041434519
S111DDB53D6E65787420706167652C204D49C1
S111DDC34E55533D7072657620706167652C75
S111DDD120616E79206F74686572206B65792D
S111DDDF2065786974732E001B5B31303B3273
S111DDED35481B5B6D1B5B4A1B5B31323B32BE
S111DDFB38484578616D696E6520496E64692B
S111DE0976696475616C204C6F636174696F97
S111DE176E731B5B31343B3238483C4144444B
S111DE25524553533E202E2E2E20666F72203F
S111DE337370656369666963206C6F63617464
S111DE41696F6E1B5B31353B3238483C4E3EF8
S111DE4F3C5245543E202E2E2E2E20666F721D
S111DE5D206E65787420616464726573731BB3
S111DE6B5B31363B3238483C52455455524EDA
S111DE793E202E2E2E2E20746F2065786974A4
S111DE870D0A000D0A1B5B6D09090941646454
S111DE95726573733A20000956616C75653A24
S111DEA320001B5B373B3333481B5B4A1B5B81
S111DEB16D1B5B316D46696C6C2F436F70798D
S111DEBF204D656E751B5B31303B3332484697
S111DECD1B5B6D696C6C204D656D6F72792066
S111DEDB426C6F636B1B5B316D1B5B31313B23
S111DEE9333248431B5B6D6F7079204D656DBD
S111DEF76F727920426C6F636B1B5B31353B9D
S111DF0533354853656C656374696F6E3F0075
S111DF131B5B31313B3332481B5B4B1B5B31D4
S111DF21353B3237481B5B6D456E74657220CC
S111DF2F5374617274696E6720416464726594
S111DF3D73733A201B5B6D1B5B376D20202035
S111DF4B201B5B31353B353148001B5B6D1BE1
S111DF595B31363B323748456E7465722045A5
S111DF676E64696E6720416464726573733A78
S111DF752020201B5B6D1B5B376D20202020BD
S111DF831B5B31363B353148001B5B6D1B5B6D
S111DF9131373B32374846696C6C2056616C60
S111DF9F75653A201B5B6D1B5B376D20201BE4
S111DFAD5B31373B333948001B5B31393B3362
S111DFBB38481B5B316D446F6E6521001B5BA3
S111DFC931303B3332481B5B4B1B5B31353B25
S111DFD73237481B5B6D456E746572205374BF
S111DFE5617274696E672041646472657373BF
S111DFF33A201B5B6D1B5B376D202020201B2A
S111E0015B31353B353148001B5B6D1B5B31D9
S111E00F363B323748456E74657220456E64A8
S111E01D696E6720416464726573733A202053
S111E02B201B5B6D1B5B376D202020201B5BD0
S111E03931363B353148001B5B6D1B5B3137C4
S111E0473B323748456E74657220546172672F
S111E055657420416464726573733A20202060
S111E0631B5B6D1B5B376D202020201B5B3187
S111E071373B353148001B5B31393B333848AF
S111E07F1B5B316D446F6E6521001B5B3130FD
S111E08D3B3235481B5B6D1B5B4A1B5B31321B
S111E09B3B3238484D6F64696679204D656DDF
S111E0A96F72792F5265676973746572204C2B
S111E0B76F636174696F6E2873291B5B3134CB
S111E0C53B3238483C414444524553533E20BC
S111E0D32E2E2E20666F7220737065636966B0
S111E0E16963206C6F636174696F6E1B5B3141
S111E0EF353B3238483C4E3E3C5245543E20B0
S111E0FD2E2E2E2E20666F72206E65787420F3
S111E10B616464726573731B5B31363B32389A
S111E119483C52455455524E3E202E2E2E2E7A
S111E12720746F20657869740D0A000D0A09D2
S111E1350909416464726573733A2000095647
S111E143616C75653A200009446F6E65000D2D
S111E15109090909001B5B373B3334481B5B8B
S111E15F4A1B5B6D1B5B316D4F7074696F6EF4
S111E16D73204D656E751B5B31313B333348B7
S111E17B431B5B6D6F6C642052657365741BEF
S111E1895B6D1B5B31323B3333481B5B316DE6
S111E197561B5B6D6563746F72204469737070
S111E1A56C61791B5B6D1B5B31333B3333487C
S111E1B31B5B316D451B5B6D4550524F4D207B
S111E1C14F7065726174696F6E731B5B6D1B2A
S111E1CF5B31343B3333481B5B316D521B5BB9
S111E1DD6D6F6D2054657374202843524329DE
S111E1EB1B5B31373B33354853656C656374F9
S111E1F9696F6E3F001B5B31313B3330481BB6
S111E2075B4B1B5B31333B3332481B5B4A528B
S111E21545534554202837464645293A2000F3
S111E2230D0A0953434920496E7465727275E1
S111E231707420202837464436293A200020F5
S111E23F200953504920496E7465727275703F
S111E24D7420202837464438293A20000D0A50
S111E25B0950756C736520492F502045646787
S111E26965202837464441293A200020200928
S111E27750756C7365204F766572666C6F7718
S111E285202837464443293A20000D0A095444
S111E293696D6572204F766572666C6F772038
S111E2A12837464445293A20002020094F2FF3
S111E2AF5020436F6D70617265203520202869
S111E2BD37464530293A20000D0A094F2F50EC
S111E2CB20436F6D7061726520342020283767
S111E2D9464532293A20002020094F2F5020BC
S111E2E7436F6D706172652033202028374626
S111E2F54534293A20000D0A094F2F502043CA
S111E3036F6D70617265203220202837464508
S111E31136293A20002020094F2F5020436F58
S111E31F6D7061726520312020283746453824
S111E32D293A20000D0A09492F50204361703F
S111E33B747572652033202028374645412929
S111E3493A2000202009492F502043617074AF
S111E357757265203220202837464543293A46
S111E36520000D0A09492F5020436170747581
S111E3737265203120202837464545293A207E
S111E381002020095265616C2054696D6520EE
S111E38F496E7420202837464630293A200073
S111E39D0D0A0949525120496E746572727559
S111E3AB707420202837464632293A2000207C
S111E3B920095849525120496E7465727275DC
S111E3C77074202837464634293A20000D0A87
S111E3D50953574920496E746572727570744D
S111E3E320202837464636293A2000202009FB
S111E3F1496C6C6567616C204F70636F6465E6
S111E3FF202837464638293A20000D0A0943E3
S111E40D4F50205761746368646F67202020AD
S111E41B2837464641293A2000202009436C48
S111E4296F636B204D6F6E69746F7220202834
S111E43737464643293A20001B5B373B3333FC
S111E445481B5B4A1B5B6D1B5B316D2045451C
S111E45350524F4D204D656E751B5B31313BB1
S111E461333148451B5B6D7261736520454580
S111E46F50524F4D20627974651B5B316D1B5A
S111E47D5B31323B333148421B5B6D756C6B77
S111E48B20457261736520454550524F4D1B6C
S111E4995B316D1B5B31333B333148571B5BEA
S111E4A76D7269746520454550524F4D2062D8
S111E4B57974651B5B316D1B5B31343B333175
S111E4C348531B5B6D6574205343492062610E
S111E4D1756420726174651B5B31373B333513
S111E4DF4853656C656374696F6E3F001B5B88
S111E4ED31373B3235481B5B6D456E746572EA
S111E4FB204164647265737320746F2045526F
S111E5094153453A201B5B6D1B5B376D202090
S111E51720201B5B31373B343948001B5B313D
S111E525373B3235481B5B6D456E74657220C2
S111E5334164647265737320746F20575249FB
S111E54154453A201B5B6D1B5B376D20202078
S111E54F201B5B31373B343948001B5B3137EE
S111E55D3B3235481B5B6D42554C4B204552FA
S111E56B41534520616C6C20353132206279B9
S111E5797465732028592F4E293F001B5B3216
S111E587313B3338481B5B316D446F6E6521A8
S111E595001B5B6D1B5B31393B333048566114
S111E5A36C756520746F2057726974653A2098
S111E5B11B5B6D1B5B376D20201B5B31393B00
S111E5BF343648001B5B373B3331481B5B4A44
S111E5CD1B5B6D1B5B316D534349204261752E
S111E5DB642052617465204D656E751B5B31C2
S111E5E9313B333248311B5B6D202E2E2E2029
S111E5F733382E34206B626175641B5B316D0A
S111E6051B5B31323B333248321B5B6D202EDF
S111E6132E2E2031392E32206B626175641B6D
S111E6215B316D1B5B31333B333248331B5B83
S111E62F6D202E2E2E2039363030206261757B
S111E63D641B5B316D1B5B31343B333248345C
S111E64B1B5B6D202E2E2E20343830302062C2
S111E6596175641B5B316D1B5B31353B3332E5
S111E66748351B5B6D202E2E2E2032343030B1
S111E67520626175641B5B31373B33354853BB
S111E683656C656374696F6E3F001B5B32311A
S111E6913B3338481B5B316D446F6E65211BB3
S111E69F5B32333B31374841646A7573742033
S111E6AD5043206261756420726174652061BF
S111E6BB6E642068697420616E79206B657945
S111E6C920746F20636F6E74696E75652E0089
S111E6D71B5B373B3236481B5B4A1B5B6D1BDB
S111E6E55B316D1B5B373B32364820202043EF
S111E6F379636C696320526564756E64616EB0
S111E701637920436865636B1B5B6D1B5B31A2
S111E70F303B323748456E7465722053746196
S111E71D7274696E6720416464726573733AA6
S111E72B201B5B376D202020201B5B31303B10
S111E739353148001B5B6D1B5B31323B3237C0
S111E74748456E74657220456E64696E6720E5
S111E755416464726573733A201B5B376D2058
S111E7632020201B5B31323B343948001B5B05
S111E7716D1B5B31343B3237484550524F4DDF
S111E77F2043524320436865636B73756D201D
S111E78D69733A201B5B376D202020201B5B34
S111E79B31343B353048001B5B6D1B5B316D28
S111E7A91B5B32303B3237485072657373206D
S111E7B7616E79206B657920746F20636F6E3C
S111E7C574696E7565001B5B373B3333481B6C
S111E7D35B4A1B5B6D1B5B316D202020527571
S111E7E16E204D656E751B5B31303B33344842
S111E7EF501B5B6D726F6772616D2052756E08
S111E7FD1B5B316D1B5B31313B333448531BC6
S111E80B5B6D7562726F7574696E652052756F
S111E8196E1B5B31353B33354853656C6563CC
S111E82774696F6E3F001B5B31353B3237481E
S111E8351B5B4B1B5B6D456E74657220537448
S111E843617274696E67204164647265737358
S111E8513A201B5B6D1B5B376D202020201BC3
S111E85F5B31353B353148001B5B31353B32B4
S111E86D36481B5B4B1B5B6D202020202020B7
S111E87B2020202052756E6E696E6721001BEE
S111E8895B31353B3236481B5B4B1B5B6D45E8
S111E8976E74657220537562726F7574696ECB
S111E8A56520416464726573733A201B5B6DD9
S111E8B31B5B376D202020201B5B31353B356D
S111E8C13248001B5B32333B3235481B5B4B45
S111E8CF1B5B6D456E746572205365742042A8
S111E8DD7265616B706F696E742041646472C1
S111E8EB6573733A201B5B6D1B5B376D202039
S111E8F920201B5B32333B353548001B5B325D
S111E907333B3235481B5B316D205768696322
S111E9156820427265616B706F696E743F20FA
S111E92328312C322C332C34291B5B6D001B45
S111E9315B32333B3235481B5B4B1B5B6D1B6B
S111E93F5B32333B3335481B5B316D53656CE3
S111E94D656374696F6E3F1B5B6D001B5B326C
S111E95B333B3235481B5B4B1B5B316D202078
S111E96920205468617420425020616C726555
S111E9776164792075736564211B5B6D001B60
S111E9855B32333B3235481B5B4B1B5B316D01
S111E9932020205468617420425020616C7270
S111E9A16561647920636C656172211B5B6D96
S111E9AF001B5B6D1B5B32333B3235481B5B38
S111E9BD4B1B5B316D20202020202020436165
S111E9CB6E27742073657420612042502074FE
S111E9D968657265211B5B6D001B5B32333B6E
S111E9E73335481B5B4B1B5B316D2052756E44
S111E9F56E696E67211B5B6D20001B5B324A4E
S111EA031B5B323B3239481B5B6D1B5B316D74
S111EA112A20363848433131204350552057CF
S111EA1F494E444F57202A1B5B353B35485067
S111EA2D433D1B5B353B3133483E1B5B373B9F
S111EA3B354820533D1B5B373B3133483E1BAF
S111EA495B393B354820593D1B5B393B31336B
S111EA57483E1B5B31303B354820583D1B5B6D
S111EA6531303B3133483E1B5B31333B354887
S111EA73413D1B5B31333B3132483D421B5B5E
S111EA8131323B3232484E205A205620431B7D
S111EA8F5B31333B3135484343523D20203D3B
S111EA9D1B5B6D1B5B353B3335481B5B316DDA
S111EAAB502C592C582C412C421B5B6D202EF4
S111EAB92E2E2E2E2E2E204D6F64696679208F
S111EAC7435055205265676973746572731B62
S111EAD55B363B3335481B5B316D541B5B6D68
S111EAE3202E2E2E2E2E2E2E2E2E2E2E2E2EAB
S111EAF12E2E205472616365204F6E652049FD
S111EAFF6E737472756374696F6E1B5B373BC4
S111EB0D3335481B5B316D471B5B6D202E2E8C
S111EB1B2E2E2E2E2E2E2E2E2E2E2E2E2E2072
S111EB29476F20746F206E6578742052545329
S111EB371B5B383B3335481B5B316D521B5B57
S111EB456D202E2E2E2E2E2E2E2E2E2E2E2E09
S111EB532E2E2E2052756E2050726F67726146
S111EB616D2066726F6D2050431B5B393B3391
S111EB6F35481B5B316D4573631B5B6D202EB7
S111EB7D2E2E2E2E2E2E2E2E2E2E2E2E2045F9
S111EB8B78697420746F204D61696E204D65A9
S111EB996E751B5B31313B3335481B5B316DB0
S111EBA74E1B5B6D202E2E2E2E2E2E2E2E2E6D
S111EBB52E2E2E2E2E2E20536574204D756CA0
S111EBC37469706C65205472616365204E7530
S111EBD16D6265721B5B31323B3335481B5B52
S111EBDF316D4D1B5B6D202E2E2E2E2E2E2EF4
S111EBED2E2E2E2E2E2E2E2E2045786563758C
S111EBFB7465204D756C7469706C65205472DD
S111EC096163651B5B31333B3335481B5B375E
S111EC176D20201B5B6D202E2E204375727223
S111EC25656E74204D756C7469706C652054B6
S111EC337261636520436F756E7420286865F6
S111EC4178291B5B31363B3239481B5B6D1B57
S111EC4F5B316D2A20425245414B504F494ED5
S111EC5D542057494E444F57202A1B5B6D1B11
S111EC6B5B31383B3548427265616B706F69EE
S111EC796E742023313D1B5B376D202020205C
S111EC871B5B6D1B5B31393B35484272656186
S111EC956B706F696E742023323D1B5B376D0C
S111ECA3202020201B5B6D1B5B31393B333579
S111ECB1481B5B316D431B5B6D6C656172200B
S111ECBF427265616B706F696E741B5B32305C
S111ECCD3B3548427265616B706F696E74204E
S111ECDB23333D1B5B376D202020201B5B6D17
S111ECE91B5B32303B3335481B5B316D531BD4
S111ECF75B6D657420427265616B706F696EAF
S111ED05741B5B32313B3548427265616B70A2
S111ED136F696E742023343D1B5B376D202026
S111ED2120201B5B6D001B5B353B38481B5BE1
S111ED2F376D001B5B353B3134481B5B6D00B8
S111ED3D1B5B373B38481B5B376D001B5B3795
S111ED4B3B3134481B5B6D001B5B393B384881
S111ED591B5B376D001B5B393B3134481B5B81
S111ED676D001B5B31303B38481B5B376D0081
S111ED751B5B31303B3134481B5B6D001B5B74
S111ED8331333B37481B5B376D001B5B31336C
S111ED913B3130481B5B376D001B5B31333B5D
S111ED9F3139481B5B376D001B5B31333B324F
S111EDAD32481B5B376D001B5B31333B333543
S111EDBB481B5B376D001B5B343B3135481B36
S111EDC95B4B1B5B343B313548001B5B313820
S111EDD73B3139481B5B376D202020201B5B2D
S111EDE531383B313948001B5B31393B313941
S111EDF3481B5B376D202020201B5B31393B11
S111EE01313948001B5B32303B3139481B5B12
S111EE0F376D202020201B5B32303B31394808
S111EE1D001B5B32313B3139481B5B376D20E3
S111EE2B2020201B5B32313B313948001B5B39
S111EE39353B38481B5B376D202020201B5BC7
S111EE47353B3848001B5B393B38481B5B37B2
S111EE556D202020201B5B393B3848001B5BDE
S111EE6331303B38481B5B376D202020201BCC
S111EE715B31303B3848001B5B31333B374884
S111EE7F1B5B376D20201B5B31333B37480093
S111EE8D1B5B31333B3130481B5B376D20205B
S111EE9B1B5B31333B313048001B5B31333B92
S111EEA93335481B5B376D20201B5B31333B38
S111EEB7333548001B5B32323B3239481B5B5B
S111EEC54B1B5B356D1B5B316D2A2A2A2A2AF2
S111EED32A205741524E494E4721202A2A2A0E
S111EEE12A2A2A1B5B6D1B5B316D1B5B3233CF
S111EEEF3B32324820494C4C4547414C2042AE
S111EEFD5245414B504F494E54204F52204F26
S111EF0B50434F44452041543A20001B5B32D2
S111EF19343B323748507265737320616E7951
S111EF27206B657920746F20636F6E74696EC1
S111EF357565001B5B32333B3234481B5B4B6B
S111EF431B5B316D425245414B504F494E54B9
S111EF5120230020454E434F554E5445524553
S111EF5F442041543A20001B5B32343B3237CD
S111EF6D48507265737320616E79206B65796C
S111EF7B20746F20636F6E74696E7565001BE1
S111EF895B32333B3234481B5B4B1B5B316DF8
S111EF972043616E27742074726163652074D8
S111EFA568726F75676820425245414B504FA9
S111EFB3494E54211B5B6D001B5B32323B3216
S111EFC134481B5B4B1B5B316D2020464154D2
S111EFCF414C204552524F52202D20535441A4
S111EFDD434B20425245414348211B5B3233D3
S111EFEB3B38482046616D6F7573204368699A
S111EFF96E6573652050726F766572623A2001
S111F00748652077686F205053482773206FA8
S111F01572204A53522773206D757374205075
S111F023554C206F72205254532E201B5B322A
S111F031343B323448536F727279202D2050D4
S111F03F7265737320616E79206B657920749D
S111F04D6F2072657365742E2E2E001B5B32CD
S111F05B333B3238481B5B4B1B5B316D4578F1
S111F06965637574696F6E2068616C7465640C
S111F07720617420525453001B5B313B37352B
S111F085481B5B4B1B5B316D496E7473211B82
S111F0935B6D001B5B324A1B5B6D1B5B303BED
S111F0A130480D0A486D6D6D2E20204C6574AC
S111F0AF2773207365652E2020596F75277610
S111F0BD65206265656E206861636B696E672D
S111F0CB204D6963726F31312E0D0A416E645F
S111F0D920796F75206A75737420646F776EEA
S111F0E76C6F6164656420612066696C652E3F
S111F0F520204D6179626520746861740D0AF3
S111F103646F776E6C6F616465642066696C7E
S111F111652069736E277420736F20696E7415
S111F11F616374206569746865722E2E2E215A
S111F12D0D0A0D0A507265737320616E79200D
S111F13B6B657920746F2072657475726E2096
S111F149746F203F000000010100000101016D
S111F1570100000101000000000101000001A0
S111F165010101000001010000010100000190
S111F173010000000001010000010101010083
S111F181000101000000000101000001010076
S111F18F000101000001010101000001010066
S111F19D000000010100000101010100000159
S111F1AB01000001010000010100000000014C
S111F1B901000001010101000001010000003D
S110F1C700010100000101FE7FD66E00FE74
S111F1D47FD86E00FE7FDA6E00FE7FDC6E00D8
S111F1E2FE7FDE6E00FE7FE06E00FE7FE26EBA
S111F1F000FE7FE46E00FE7FE66E00FE7FE808
S110F1FE6E00FE7FEA6E00FE7FEC6E00FEE8
S111F20B7FEE6E00FE7FF06E00FE7FF26E005E
S111F219FE7FF46E00FE7FF66E00FE7FF86E40
S10EF22700FE7FFA6E00FE7FFC6E000C
S111FE0030EC09CE7FAD188F4F1AAC002717D7
S110FE0E08084C8104270220F2CEFE54BDEA
S111FE1BCB92188FBDCB857EFE4D6F006F011C
S111FE29CE7FB5163AA60018A700CEFE92BDF5
S10FFE37CB92178B31BDCB51CEFEA1BD88
S10EFE43CB92188FBDCB857EFE4DCE08
S111FE4EFEB3BDCB92390A0D2A2A2A2A2A2A8B
S111FE5C205741524E494E4721202A2A2A2A75
S111FE6A2A2A0A0D52554E4157415920425240
S111FE7845414B504F494E5420454E434F5583
S111FE864E54455245442041543A20000A0D82
S111FE94425245414B504F494E54202300200A
S111FEA2454E434F554E54455245442041545D
S111FEB03A20000A0D205461736B09537461EB
S111FEBE74650943432041202042202058202F
S111FECC2020205920202020532020202050C8
S108FEDA430A0D2000A5
S109FFD6F1CEF1D3F1D8D5
S109FFDCF1DDF1E2F1E7A2
S109FFE2F1ECF1F1F1F66F
S109FFE8F1FBF200F2053A
S109FFEEF20AF20FF21406
S109FFF4F219F21EF223D3
S109FFFAF228F22DC00004
S9030000FC
